S01A000064656D6F70726F675F73746D3332673037312E7372656396
S3150800200000900020E54300083544000835440008E0
S3150800201000000000000000000000000000000000B2
S315080020200000000000000000000000003544000821
S315080020300000000000000000354400086544000860
S31508002040354400083544000835440008354400087E
S31508002050354400083544000835440008354400086E
S31508002060354400083544000835440008354400085E
S31508002070354400083544000835440008354400084E
S31508002080354400083544000835440008354400083E
S31508002090354400083544000835440008354400082E
S315080020A0354400083544000835440008354400081E
S315080020B0354400083544000835440008EE11AA5591
S315080020C010B5064C2378002B07D1054B002B02D000
S315080020D0044800E000BF0123237010BD0C00002057
S315080020E000000000C8440008044B10B5002B03D0BC
S315080020F00349044800E000BF10BDC04600000000C8
S3150800210010000020C8440008002243088B4274D3FC
S3150800211003098B425FD3030A8B4244D3030B8B42DA
S3150800212028D3030C8B420DD3FF22090212BA030CE3
S315080021308B4202D31212090265D0030B8B4219D3C4
S3150800214000E0090AC30B8B4201D3CB03C01A5241E4
S31508002150830B8B4201D38B03C01A5241430B8B422C
S3150800216001D34B03C01A5241030B8B4201D30B0315
S31508002170C01A5241C30A8B4201D3CB02C01A52413C
S31508002180830A8B4201D38B02C01A5241430A8B42FF
S3150800219001D34B02C01A5241030A8B4201D30B02E8
S315080021A0C01A5241CDD2C3098B4201D3CB01C01A02
S315080021B0524183098B4201D38B01C01A524143090C
S315080021C08B4201D34B01C01A524103098B4201D3FA
S315080021D00B01C01A5241C3088B4201D3CB00C01A67
S315080021E0524183088B4201D38B00C01A52414308DF
S315080021F08B4201D34B00C01A5241411A00D2014604
S31508002200524110467047FFE701B5002000F006F876
S3150800221002BDC0460029F7D076E770477047C0462A
S31508002220002B11D1002A0FD1002900D1002802D095
S315080022300021C943081C07B4024802A140180290AD
S3150800224003BDC046D9FFFFFF03B4684601B502982F
S3150800225000F006F8019B9E4602B00CBC7047C046CB
S31508002260F0B557464E464546DE46E0B5040083B00F
S315080022700D00924699468B422FD82CD04946504697
S3150800228000F0AEF829000600200000F0A9F8331A7D
S315080022909846203B9B4600D574E053465A469340E1
S315080022A01F005346424693401E00AF4229D826D007
S315080022B05B46A41BBD41002B00DA79E0002200230F
S315080022C00092019301235A46934001930123424603
S315080022D09340009319E08242D0D90022002300924D
S315080022E001930C9B002B01D01C605D60009801993E
S315080022F003B03CBC90469946A246AB46F0BDA34205
S31508002300D6D900220023009201934346002BE8D039
S31508002310FB0772081A4346467B080EE0AB4201D11A
S31508002320A2420CD8A41A9D41012024196D4100210E
S31508002330013E24184D41002E06D0AB42EED9013E8F
S3150800234024196D41002EF8D15B46009801990019B1
S315080023506941002B22DB2B005A46D3402A0044460B
S31508002360E2401C005B461500002B2CDB26009E4035
S31508002370330026004746BE403200801A9941009035
S315080023800191AEE7424620239B1A5246DA4041465F
S3150800239013004A468A4017001F4382E74246202315
S315080023A09B1A2A0046469A402300F3401343D5E772
S315080023B04246202300219B1A002200910192012205
S315080023C0DA40019282E74246202326009B1ADE4025
S315080023D02F00B446974066463B003343C9E7C046DC
S315080023E010B5002903D100F007F8203002E0081CD8
S315080023F000F002F810BDC0461C2101231B049842B8
S3150800240001D3000C10391B0A984201D3000A083977
S315080024101B09984201D30009043902A2105C40182E
S315080024207047C046040302020101010100000000D2
S315080024300000000010B50A480A4B0360E1231B029E
S31508002440436000238360C360036183610C22426199
S31508002450C361802212010262436201F0C9FE10BD07
S31508002460280000200044004010B501000023012286
S31508002470044801F0D7FD002801D0002010BD013026
S31508002480FCE7C0462800002010B5FFF7D3FF10BDB3
S31508002490BFF34F8F034A044BDA60BFF34F8FC04632
S315080024A0FDE7C0460400FA0500ED00E010B5214B33
S315080024B01B78002B16D12048FFF7D6FF012800D03D
S315080024C010BD1D4B1B78013BDBB23F2BF8D801F042
S315080024D0C5FF1A4B18600122164B1A700022184BBA
S315080024E01A70EDE7164B1B7801331348C018FFF72F
S315080024F0BBFF01280AD001F0B1FF104B1B686433FB
S315080025009842DDD900220B4B1A70D9E70C4A13788A
S315080025100133DBB21370084A12789342D0D10021F6
S31508002520044A1170044A5278FF2AC9D1022BC7D12E
S31508002530FFF7AEFFF5000020B4000020F8000020E9
S31508002540F600002010B5FFF7B1FF10BD10B5002248
S315080025502021A020C00500F099F910BD10B501F0A2
S315080025607DFF04000F4B1B68C31AF422FF32934207
S315080025700ED90D4B1B78002B0BD1F33AFF3A0A4BB9
S315080025801A702021A020C00500F080F9054B1C60B8
S3150800259010BD0022044B1A702021A020C00500F0AF
S315080025A075F9F3E700010020FC00002010B50400CF
S315080025B0104B1968002901D1012010BDFA208000AE
S315080025C0FFF7A2FD01000C4B1868FFF79DFD00F010
S315080025D06FF800280CD1032C01D90120EDE7002261
S315080025E02100013800F032F8044B1C600020E4E7B3
S315080025F00120E2E700000020080000200400002077
S3150800260010B5084A116880235B000B43136000204D
S31508002610FFF7CCFF041E02D00124200010BD01F0F4
S3150800262091FEFAE700200240034A13680349096845
S315080026305B1813607047C0460401002000000020A4
S31508002640014B18687047C0460401002070B5002881
S3150800265011DB8308144DC0339B005C5903221040DC
S31508002660C000FC3216008640B44389010A40824005
S3150800267022435A5170BDC0B20F230340083B9B0842
S3150800268006339B00094A944663445D68032210405A
S31508002690C000FF2422008240954389010C408440F3
S315080026A02C435C60E6E7C04600E100E000ED00E090
S315080026B001380A4B98420FD8094A50600948036AFC
S315080026C01B021B0AC02109060B4303620023936001
S315080026D007331360002070470120FCE7FFFFFF0067
S315080026E010E000E000ED00E0042805D0054A136874
S315080026F004218B4313607047024A136804210B4375
S315080027001360F8E710E000E0704710B5FFF7FCFF2C
S3150800271010BD0000F0B5C64600B5002379E0DF0815
S315080027200837BF003E5807251D40AD000F24AC40B2
S31508002730A6430C69AC40250035433D5079E08568D1
S3150800274064462540CE68BE403543856045682C0002
S315080027504546AC434D682E09012535409D402C431E
S315080027604460C46865462C408D68BD402C43C460EF
S315080027704C68E4004CD59C0825001835AD003F4E42
S31508002780AE5903251D40ED000F27AF40BE43A027D5
S31508002790FF05B84268D03A4FB84267D0394FB842B9
S315080027A066D0394FB8425DD00527AF403D00354366
S315080027B0324E1834A400A55180243559D443260036
S315080027C02E404F68FF0301D515432E002B4D802759
S315080027D0EE518426AD592E0026404F68BF0301D519
S315080027E015432E00254D8427EE512D682E002640D0
S315080027F04F68FF0201D515432E00204D2E606D68E7
S315080028002C404E68B60201D52A4314001B4A546070
S3150800281001330A681400DC402CD001249C40A046F1
S315080028202240F5D04D68022D00D178E7122D00D14F
S3150800283075E706685F0003252C00BC40E443A44600
S3150800284026404C682540BD40354305604D686E1EE0
S31508002850012E00D873E7112D00D170E7122D00D094
S315080028607FE76CE70327A0E700279EE701279CE799
S3150800287002279AE704BC9046F0BDC04600180240FD
S315080028800004005000080050000C0050002A01D136
S31508002890816270478161FCE710B5104A13681049D8
S315080028A00B400343136080239B00984201D000200D
S315080028B010BD0C4B1A6853009B1858000A49FFF7BD
S315080028C023FC0130054B5B695B0503D5002803D063
S315080028D00138F7E70020EBE70320E9E7007000403E
S315080028E0FFF9FFFF0800002040420F0070B582B0D4
S315080028F0041E00D142E20368DB0739D5C34A916852
S3150800290038230B40D16803220A40102B26D0082B07
S3150800291026D063688022520293427FD0A022D20238
S31508002920934200D181E0B94B1A68B9490A401A6046
S315080029301A68B8490A401A606368002B00D180E01B
S31508002940FFF77EFE0500B14B1B689B0310D4FFF70B
S3150800295077FE401B6428F6D903201AE2032AD6D14B
S31508002960AA4B1B689B0303D56368002B00D107E2BB
S3150800297023689B0731D5A54A936838210B40D1684F
S3150800298003220A40102B6AD0002B6BD19F4A12688B
S31508002990520503D5E268002A00D1F3E19B48426854
S315080029A09D490A40616909020A434260002B0DD11C
S315080029B003689A490B4021690B4303600368DB0AE5
S315080029C007221A40964BD340964A1360964B1868CE
S315080029D0FFF7ECFD002800D0D6E123681B0700D4DA
S315080029E081E08A4B9A6838231340182B73D0A36961
S315080029F0002B00D194E0854A136E01210B43136620
S31508002A00FFF71EFE0500814B1B6E9B076BD4FFF775
S31508002A1017FE401B0228F6D90320BAE17B4A116843
S31508002A2080235B020B43136086E7784B1968802284
S31508002A30D2020A431A601968802252020A431A60AF
S31508002A407AE7FFF7FDFD0500704B1B689B038FD5E2
S31508002A50FFF7F6FD401B6428F6D9032099E1022A00
S31508002A6092D193E7E368002B22D0684A13686B4932
S31508002A700B4021690B431360116880235B000B43ED
S31508002A801360FFF7DDFD0500604B1B685B0506D488
S31508002A90FFF7D6FD401B0228F6D9032079E15B49EA
S31508002AA04B685D4A13406269120213434B6094E710
S31508002AB0564A13685D490B401360FFF7C1FD0500D0
S31508002AC0524B1B685B0588D5FFF7BAFD401B0228E9
S31508002AD0F6D903205DE14D4B1B6E9B0703D5A36911
S31508002AE0002B00D152E123685B0700D4A6E0474BD0
S31508002AF09A6838231340202B25D0444BDB6BDB0028
S31508002B002AD40123002B29D0404AD16B80204005C6
S31508002B100143D163D36B03400193019B01251EE05A
S31508002B203A4A136E01218B431366FFF789FD0500A8
S31508002B30364B1B6E9B07D6D5FFF782FD401B022836
S31508002B40F6D9032025E1314BDB6D9B0776D5A368C3
S31508002B50002B73D101201CE10023D3E70025344B59
S31508002B601B68DB051FD5A368012B30D0052B34D095
S31508002B70264BDA6D01218A43DA65DA6D03318A4319
S31508002B80DA65A368002B32D0FFF75AFD06001F4B03
S31508002B90DB6D9B0750D4FFF753FD801B254B9842EE
S31508002BA0F5D90320F5E0224A116880235B000B4320
S31508002BB01360FFF745FD06001D4B1B68DB05D2D4E5
S31508002BC0FFF73EFD801B0228F6D90320E1E00F4AF5
S31508002BD0D36D01210B43D365D3E70C4BDA6D042182
S31508002BE00A43DA65DA6D03390A43DA65C9E7FFF796
S31508002BF027FD0600054BDB6D9B071DD5FFF720FD5E
S31508002C00801B0C4B9842F5D90320C2E00010024005
S31508002C10FFFFFEFFFFFFFBFFFF80FFFFFFC7FFFF72
S31508002C200024F4000800002004000020FFFEFFFF37
S31508002C300070004088130000012D26D0E369002BA0
S31508002C4000D1A5E0564A916838220A40102A63D076
S31508002C50022B20D0524B1A6852490A401A60DA6889
S31508002C6003218A43DA60DA684F490A40DA60FFF7D7
S31508002C70E7FC04004A4B1B689B014BD5FFF7E0FCB9
S31508002C80001B0228F6D9032083E0454AD36B47493F
S31508002C900B40D363D2E7424A136842490B4013609C
S31508002CA0FFF7CEFC05003E4B1B689B0106D5FFF7D8
S31508002CB0C7FC401B0228F6D903206AE0384AD368C5
S31508002CC03B491940236A606A0343A06A000203432A
S31508002CD0E06A0343206B0343606B03430B43D360F3
S31508002CE0116880235B040B431360D16880235B055E
S31508002CF00B43D360FFF7A4FC0400294B1B689B0118
S31508002D0006D4FFF79DFC001B0228F6D9032040E0F5
S31508002D1000203EE000203CE0012B3CD0204BDA6846
S31508002D2003231340216A8B4201D0012031E070232E
S31508002D301340616A8B4201D001202AE0FE21C901B5
S31508002D401140A36A1B02994201D0012021E0F82311
S31508002D509B031340E16A8B4201D0012019E0E0236E
S31508002D601B051340216B8B4201D0012011E0520F45
S31508002D705207636B9A4210D001200AE0012008E04E
S31508002D80012006E0012004E0012002E0012000E025
S31508002D90002002B070BD0120FBE70020F9E7C0461D
S31508002DA000100240FFFFFFFEFFFFFEEEFFFFFFEFF2
S31508002DB08C80C11110B52B4B9B6838221A4219D04A
S31508002DC0284B9A6838231340082B46D0254B9A6817
S31508002DD038231340102B18D0224B9A6838231340F7
S31508002DE0202B3CD01F4B9A6838231340182B31D020
S31508002DF0002009E01B4B1A68D20A07231340012159
S31508002E0099401948FFF780F910BD164AD1680D3B5D
S31508002E100B40D2681209072111400131032B0FD14B
S31508002E201248FFF771F90F4BDA68120A7F2313402D
S31508002E3058430C4BD968490F0131FFF765F9E3E7A9
S31508002E400948FFF761F9074BDA68120A7F2313402E
S31508002E505843EEE7FA20C001D6E70448D4E78020B5
S31508002E600002D1E7001002400024F40000127A00A4
S31508002E7070B504000D00002800D1AAE0574B1A6867
S31508002E80072313408B4221D323689A070ED55B0785
S31508002E9005D5534A9168E023DB010B439360504AFA
S31508002EA0936850490B40A1680B4393602368DB077E
S31508002EB054D56368012B20D0022B3BD0002B3FD181
S31508002EC0474A126852051CD401206AE0434A13682F
S31508002ED007218B432B431360FFF7B2FB06003F4BDA
S31508002EE01A68072313409D42CED0FFF7A9FB801B23
S31508002EF03D4B9842F3D9032053E0394A12689203AE
S31508002F0069D537498A680720824313438B60FFF7E0
S31508002F1097FB0600324B9B6838221A406368DB0031
S31508002F209A421BD0FFF78CFB801B2F4B9842F1D996
S31508002F30032036E02A4A12689201E2D4012030E0E2
S31508002F40032B05D0264AD26D9207DAD4012028E051
S31508002F50234A126E9207D4D4012022E01F4B1A6826
S31508002F60072313409D421DD323685B0706D51C4AD9
S31508002F7093681E490B40E1680B439360FFF71AFFFD
S31508002F80174B9A68120A0F2313409B00184A9A583F
S31508002F901F231340D840174B1860174B1868FFF7C4
S31508002FA005FB70BD0D4A136807218B432B4313603D
S31508002FB0FFF746FB0600094B1A68072313409D4294
S31508002FC0D2D0FFF73DFB801B074B9842F3D903206D
S31508002FD0E7E70120E5E70120E3E7C04600200240D5
S31508002FE000100240FFF0FFFF88130000FF8FFFFF6D
S31508002FF0E04400080800002004000020014B18687F
S315080030007047C0460800002010B5FFF7F7FF064BCB
S315080030109A68120B072313409B00044A9A581F23E9
S315080030201340D84010BDC046001002402045000895
S31508003030F0B583B0040003689B0360D5804BDB6B57
S31508003040DB001ED47E4AD16B802040050143D16344
S31508003050D36B03400193019B01267A4A11688023AA
S315080030605B000B431360FFF7EBFA0500754B1B6813
S31508003070DB0508D4FFF7E4FA401B0228F6D9032536
S3150800308002E00026E9E70025002D21D16C4BDB6D17
S31508003090C0229200134010D0226B93420DD0684A8A
S315080030A0D36D69490B40D06D802149020143D16532
S315080030B0D16D66480140D165D365DB0710D4002D74
S315080030C006D15F4AD36D60490B40216B0B43D3652C
S315080030D0012E15D15A4AD36B5D490B40D3630FE0D5
S315080030E0FFF7AEFA0700564BDB6D9B07E7D4FFF7F1
S315080030F0A7FAC01B574B9842F5D90325DFE70025E9
S315080031002368DB0706D54E4A536D03218B43616856
S315080031100B43536523689B0706D5494A536D0C2113
S315080031208B43A1680B43536523689B0606D5444A1F
S31508003130536D49490B40E1680B43536523689B056A
S3150800314006D53F4A536D45490B40A1690B43536564
S3150800315023685B0506D53A4A536D41490B40E16938
S315080031600B43536523685B0606D5354A536D3D49BF
S315080031700B4021690B43536523685B040BD5304A22
S31508003180536D9B009B08216A0B4353658023DB051F
S31508003190226A9A4239D023681B0306D5284A536DFA
S315080031A040218B43616A0B43536523689B020BD509
S315080031B0234A536D2C490B40A16A0B435365802360
S315080031C0DB03A26A9A4227D023685B020BD51C4A06
S315080031D0536D26490B40E16A0B43536580235B0414
S315080031E0E26A9A421FD023681B050BD5144A536D11
S315080031F01F490B4061690B43536562698023DB01F4
S315080032009A4215D0280003B0F0BD0D4AD168802334
S315080032105B020B43D360BEE7094AD16880235B048F
S315080032200B43D360D0E7064AD1680B43D360DAE78D
S31508003230034AD16880235B020B43D360E2E7C046AA
S315080032400010024000700040FFFCFFFFFFFFFEFF7A
S31508003250FFFFFFEF88130000FFF3FFFFFFFFF3FFF9
S31508003260FFFFCFFFFFCFFFFFFFFFBFFFFFFFFFFE01
S31508003270FF3FFFFF70470000F8B505000168836847
S315080032800269134342691343C2691343426E1343E7
S315080032900A68BC48024013430B602A685368BA4957
S315080032A00B40E9680B435360AB692A68B7498A4201
S315080032B001D0296A0B439168B54801400B439360D6
S315080032C02A68D36A0F218B43696A0B43D3622B683A
S315080032D0B04A93425CD0B04A93426DD0AF4A93420B
S315080032E000D19EE0AE4A934200D19CE0A74A9342A1
S315080032F077D01026A54A934200D198E080231B0276
S31508003300EA699A4200D167E3022E01D100F011FD65
S3150800331001D800F0B9FC042E01D100F046FD082EB4
S3150800332001D000F0ACFD6B6A002B01D100F080FDE6
S31508003330012B01D100F088FD022B01D100F087FD99
S31508003340032B01D100F086FD042B01D100F084FD8A
S31508003350052B01D100F083FD062B01D100F081FD7C
S31508003360072B01D100F07FFD082B01D100F07EFD6F
S31508003370092B01D100F07DFD0A2B01D100F07CFD5F
S315080033800B2B01D100F052FD8020000200F052FD07
S31508003390844A516D03220A40012A09D0002A05D021
S315080033A0022A3AD0032A05D01026A3E70026A1E769
S315080033B004269FE708269DE77A4A516D0C220A40A3
S315080033C0042A0AD005D9082A29D00C2A07D10826A2
S315080033D090E7002A03D100268CE704268AE7102600
S315080033E088E7704A526DC02109010A408021C90048
S315080033F08A420ED009D9802109018A4215D0C021F6
S3150800340009018A4207D1082674E7002A03D1002653
S3150800341070E704266EE710266CE702266AE702269E
S3150800342068E7002666E7002664E7022662E7022EBA
S3150800343000D1C1E02ED9042E00D1DCE0082E00D040
S3150800344015E16B6A002B00D135E1012B00D136E17D
S31508003450022B00D137E1032B00D138E1042B00D130
S3150800346038E1052B00D139E1062B00D139E1072BCC
S3150800347000D139E1082B00D13AE1092B00D13BE113
S315080034800A2B00D13CE10B2B00D1EDE08020000295
S31508003490002426E0002E00D0E9E0FFF7B5FD6B6AB0
S315080034A0002B1AD0012B60D0022B60D0032B60D0E2
S315080034B0042B60D0052B60D0062B60D0072B73D069
S315080034C0082B73D0092B73D00A2B73D00B2B01D082
S315080034D0012103E08021490000E00121FEF714FEE6
S315080034E00024002801D100F006FC6A6853009B18E6
S315080034F0984201D200F0C6FC1303984201D900F0A5
S31508003500C3FC022E00D15DE100D8FDE0042E00D1F7
S315080035109FE1082E00D05CE26B6A002B00D128E2FE
S31508003520012B00D130E2022B00D131E2032B00D16E
S3150800353032E2042B00D132E2052B00D133E2062B0E
S3150800354000D133E2072B00D133E2082B00D134E255
S31508003550092B00D135E20A2B00D136E20B2B00D11C
S3150800356003E280263604002706E20221B6E7042194
S31508003570B4E70621B2E70821B0E70A21AEE70C2135
S31508003580ACE7C046F369FFCFFFCFFFFF00800040DE
S31508003590FFF4FF1100380140004400400048004095
S315080035A0004C004000100240102197E7202195E7C3
S315080035B0402193E7802191E76B6A002B5AD0012BB3
S315080035C05BD0022B5CD0032B5DD0042B5ED0052B81
S315080035D05FD0062B60D0072B61D0082B62D0092B51
S315080035E063D00A2B64D00B2B02D0AB48002478E7B3
S315080035F0AA48002475E7FFF7DDFB6B6A002B1AD093
S31508003600012B1DD0022B1DD0032B1DD0042B1DD042
S31508003610052B1DD0062B1DD0072B1DD0082B1DD022
S31508003620092B1DD00A2B1DD00B2B01D0012103E03D
S315080036308021490000E00121FEF766FD002450E7DD
S315080036400221F9E70421F7E70621F5E70821F3E760
S315080036500A21F1E70C21EFE71021EDE72021EBE73E
S315080036604021E9E78021E7E78020002439E70020A8
S31508003670012436E78848002433E78948002430E7E0
S31508003680884800242DE7884800242AE7874800242C
S3150800369027E78748002424E78648002421E7864848
S315080036A000241EE7854800241BE78548002418E700
S315080036B08448002415E780200002002411E78020B2
S315080036C0C00100240DE780208001002409E77E4818
S315080036D0002406E780204001002402E77B480024F6
S315080036E0FFE67B480024FCE6802000010024F8E67B
S315080036F08020C0000024F4E6802080000024F0E644
S31508003700802040000024ECE6002E00D061E1FFF79F
S315080037107BFC6B6A002B1CD0012B35D0022B36D0D4
S31508003720032B37D0042B38D0052B39D0062B3AD0AB
S31508003730072B3BD0082B3CD0092B3DD00A2B3ED07B
S315080037400B2B02D00122002305E080225200002321
S3150800375001E0012200230021FEF762FD060E0B029E
S31508003760334302026E6870080021801859413200FE
S315080037700023FEF755FD574A574BC318934200D905
S3150800378084E32B68D860B6E202220023E3E704222A
S315080037900023E0E706220023DDE708220023DAE714
S315080037A00A220023D7E70C220023D4E7102200239D
S315080037B0D1E720220023CEE740220023CBE7802250
S315080037C00023C8E76B6A002B1BD0012B23D0022BE2
S315080037D024D0032B25D0042B26D0052B27D0062B47
S315080037E028D0072B29D0082B2AD0092B2BD00A2B17
S315080037F02CD00B2B02D0394E002704E0264E00278A
S3150800380001E0364E0027500800218019794100232F
S31508003810FEF706FDAFE7324E0027F4E7314E0027E4
S31508003820F1E7314E0027EEE7304E0027EBE7304E42
S315080038300027E8E72F4E0027E5E72F4E0027E2E7A7
S315080038402E4E0027DFE72E4E0027DCE72D4E0027F9
S31508003850D9E7FFF7AFFA6B6A002B55D0012B66D074
S31508003860022B67D0032B68D0042B69D0052B6AD0AE
S31508003870062B6BD0072B6CD0082B6DD0092B6ED07E
S315080038800A2B6FD00B2B02D0012200233EE08022A8
S31508003890520000233AE0C0460024F40024F4000055
S315080038A000127A0000093D00AAB0280080841E0094
S315080038B0006A18005558140040420F0020A107005E
S315080038C090D0030048E8010055150000CC0C000014
S315080038D0AA0A0000FFFC0F0000FDFFFF000024F409
S315080038E00000127A0000093D00AAB0280080841E54
S315080038F000006A18005558140040420F0020A1071E
S315080039000090D0030048E801012200230021FEF7B9
S3150800391087FC060E0B02334302026E68700800210C
S315080039208018594132000023FEF77AFC23E7022269
S315080039300023EBE704220023E8E706220023E5E755
S3150800394008220023E2E70A220023DFE70C220023ED
S31508003950DCE710220023D9E720220023D6E74022FD
S315080039600023D3E780220023D0E7802636020027EB
S3150800397002E0802636040027500800218019794184
S315080039800023FEF74DFCF6E68026F6030027F3E74C
S315080039908026B6030027EFE7A84E0027ECE7802627
S315080039A076030027E8E7A64E0027E5E7A54E002799
S315080039B0E2E7802636030027DEE78026F6020027A0
S315080039C0DAE78026B6020027D6E7802676020027A1
S315080039D0D2E701240020CEE6022E00D183E02DD9BD
S315080039E0042E00D1BBE0082E00D024E16B6A002B20
S315080039F000D1F9E0012B00D102E1022B00D102E14E
S31508003A00032B00D102E1042B00D101E1052B00D1E3
S31508003A1001E1062B00D100E1072B00D1FFE0082BBE
S31508003A2000D1FFE0092B00D1FFE00A2B00D1FFE00F
S31508003A300B2B00D1D5E080204002D7E0002E00D025
S31508003A40F9E0FFF7E1FA6B6A002B1AD0012B36D0A2
S31508003A50022B36D0032B36D0042B36D0052B36D086
S31508003A60062B36D0072B36D0082B36D0092B36D066
S31508003A700A2B36D00B2B01D0012103E08021490007
S31508003A8000E00121FEF740FB40006B685B08C018A8
S31508003A906968FEF739FB0004000C00246A4A030033
S31508003AA0103B934200D9F3E10F2302009A43130017
S31508003AB040080722104018432B68D8601BE10221F2
S31508003AC0E0E70421DEE70621DCE70821DAE70A2138
S31508003AD0D8E70C21D6E71021D4E72021D2E74021E8
S31508003AE0D0E78021CEE76B6A002B19D0012B22D0B4
S31508003AF0022B22D0032B22D0042B22D0052B22D036
S31508003B00062B22D0072B22D0082B22D0092B22D015
S31508003B100A2B22D00B2B01D04C4802E04C4800E07F
S31508003B204A486B685B08C0186968FEF7EDFA000436
S31508003B30000C0024B2E74748F3E74748F1E747484F
S31508003B40EFE74748EDE74748EBE74748E9E74748DF
S31508003B50E7E74748E5E74748E3E74748E1E7FFF788
S31508003B6029F96B6A002B1AD0012B26D0022B26D0F6
S31508003B70032B26D0042B26D0052B26D0062B26D0A1
S31508003B80072B26D0082B26D0092B26D00A2B26D081
S31508003B900B2B01D0012103E08021490000E001211F
S31508003BA0FEF7B2FA40006B685B08C0186968FEF752
S31508003BB0ABFA0004000C002470E70221F0E70421A8
S31508003BC0EEE70621ECE70821EAE70A21E8E70C21F7
S31508003BD0E6E71021E4E72021E2E74021E0E780213B
S31508003BE0DEE78020400001E0802040026B685B0829
S31508003BF0C0186968FEF788FA0004000C00244DE72F
S31508003C0080200002F2E78020C001EFE71B48EDE7BD
S31508003C1080208001EAE71A48E8E71A48E6E78020A4
S31508003C204001E3E780200001E0E78020C000DDE7EF
S31508003C3080208000DAE7012400202FE700551500D0
S31508003C4000CC0C0000AA0A00EFFF00000048E801BB
S31508003C5048E801000024F40000127A00546151007B
S31508003C6000093D0000D43000AAB0280080841E0058
S31508003C7040420F0020A1070090D00300AA2A0000A6
S31508003C809819000054150000002E00D0F7E0FFF741
S31508003C90BBF96B6A002B1AD0012B36D0022B36D013
S31508003CA0032B36D0042B36D0052B36D0062B36D030
S31508003CB0072B36D0082B36D0092B36D00A2B36D010
S31508003CC00B2B01D0012103E08021490000E00121EE
S31508003CD0FEF71AFA6B685B08C0186968FEF714FAEB
S31508003CE00004000C00246C4A0300103B934200D9E0
S31508003CF0D0E02B68D86001236A22AB52023AAB5255
S31508003D000023EB662B672000F8BD0221E0E70421BB
S31508003D10DEE70621DCE70821DAE70A21D8E70C21E5
S31508003D20D6E71021D4E72021D2E74021D0E7802129
S31508003D30CEE76B6A002B19D0012B22D0022B22D09A
S31508003D40032B22D0042B22D0052B22D0062B22D0DF
S31508003D50072B22D0082B22D0092B22D00A2B22D0BF
S31508003D600B2B01D04D4802E04D4800E04B486B68EC
S31508003D705B08C0186968FEF7C7F90004000C002440
S31508003D80B1E74848F3E74848F1E74848EFE74848C5
S31508003D90EDE74848EBE74848E9E74848E7E7484891
S31508003DA0E5E74848E3E74848E1E7FFF703F86B6AC1
S31508003DB0002B1AD0012B25D0022B25D0032B25D07A
S31508003DC0042B25D0052B25D0062B25D0072B25D04F
S31508003DD0082B25D0092B25D00A2B25D00B2B01D053
S31508003DE0012103E08021490000E00121FEF78CF95A
S31508003DF06B685B08C0186968FEF786F90004000C52
S31508003E00002470E70221F1E70421EFE70621EDE738
S31508003E100821EBE70A21E9E70C21E7E71021E5E7A6
S31508003E202021E3E74021E1E78021DFE7802001E068
S31508003E30802000026B685B08C0186968FEF764F9A1
S31508003E400004000C00244EE78020C001F2E7802021
S31508003E508001EFE71D48EDE780204001EAE71C48AE
S31508003E60E8E71C48E6E780200001E3E78020C00079
S31508003E70E0E780208000DDE780204000DAE70124C3
S31508003E80002030E7012436E7012434E7012432E72D
S31508003E90012430E701242EE7EFFF00000024F40098
S31508003EA024F4000000127A0000093D00AAB0280098
S31508003EB080841E00006A18005558140040420F00FE
S31508003EC020A1070090D0030048E80100551500001E
S31508003ED0CC0C0000AA0A0000836ADB0706D5026834
S31508003EE053682C490B40C16A0B435360836A9B078E
S31508003EF006D50268536828490B40016B0B4353608B
S31508003F00836A5B0706D50268536824490B40416BF0
S31508003F100B435360836A1B0706D50268536820491A
S31508003F200B40816B0B435360836ADB0606D5026838
S31508003F3093681C490B40C16B0B439360836A9B06CD
S31508003F4006D50268936818490B40016C0B439360C9
S31508003F50836A5B060BD50268536814490B40416CAB
S31508003F600B43536080235B03426C9A420AD0836AF0
S31508003F701B0606D5026853680D490B40C16C0B43F6
S31508003F8053607047026853680A490B40816C0B43BB
S31508003F905360ECE7FFFFFDFFFFFFFEFFFFFFFBFFA0
S31508003FA0FF7FFFFFFFEFFFFFFFDFFFFFFFFFEFFFD3
S31508003FB0FFFFF7FFFFFF9FFFF0B5C64600B50500F8
S31508003FC00F0016009846069C2B68DB693A009A4350
S31508003FD013005A425341B3421ED1631CF4D0FEF774
S31508003FE02FFB4346C01A844201D3002CECD12A6821
S31508003FF013680B490B4013602A689368A331FF3195
S315080040008B43936020238022AB500432AB500022AE
S315080040105C33EA54032000E0002004BC9046F0BD5F
S315080040205FFEFFFFF0B5CE4600B584B004000F0072
S3150800403016001D008423C358202B04D0022004B088
S3150800404004BC9146F0BD002900D191E0002A00D1B8
S3150800405090E080235B0182689A4205D07C23E35C6A
S31508004060012B08D10220EAE70369002BF6D1CB071A
S31508004070F4D50120E3E701227C23E25400220C3325
S31508004080E2502232043BE250FEF7DAFA03905C2350
S31508004090E6520233E652A36880225201934208D0C0
S315080040A0002B15D12269002A0ED1FF216032A152B8
S315080040B015E02269002A03D130496032A1520EE088
S315080040C0FF216022A1520AE07F216022A15206E068
S315080040D08022520593420BD000216022A152602211
S315080040E0A65A8022520193420DD00023994620E019
S315080040F02269002A03D17F216032A152EFE73F21CE
S315080041006022A152EBE72369002B02D000239946CF
S315080041100FE0B94600270CE023685B6A33404A463D
S31508004120138002239C46E1445E22A35A013B9BB2BC
S31508004130A3525E23E35A9BB2002B11D00095039B32
S31508004140002220212000FFF737FF002814D1002F76
S31508004150E2D023685B6AF2B213403B700137E3E7AB
S3150800416020228433E2500022083BE254002066E70E
S31508004170012064E7012062E7032060E7FF010000F1
S3150800418030B583B0040000228823C250FEF758FADF
S31508004190050023681B681B070ED423681B685B078A
S315080041A017D420238022A3500432A35000225C3364
S315080041B0E254002003B030BD0C4B009303000022EC
S315080041C0802189032000FFF7F7FE0028E5D00320A9
S315080041D0F0E7064B00932B0000228021C90320003C
S315080041E0FFF7EAFE0028DCD00320E3E7FFFFFF0124
S315080041F010B5041E30D08023C358002B22D02422A9
S315080042008023E2502268136801218B431360200043
S31508004210FFF732F8012814D0A36A002B18D12268B8
S3150800422053680E490B405360226893682A218B43D2
S3150800423093602268136829390B4313602000FFF73F
S315080042409FFF10BD00227C33C254FFF713F8D6E750
S315080042502000FFF741FEE2E70120F2E7FFB7FFFF84
S3150800426080221205014B9A607047C04600ED00E0B7
S31508004270014B024A9A60704700ED00E000200008F2
S3150800428000B5A1B03822002112A800F015F91022B5
S3150800429000210EA800F010F93422002101A800F030
S315080042A00BF980208000FEF7F7FA0223129380228A
S315080042B052001592002216924032179219931A93B9
S315080042C02E331B931C9280239B021D9380239B04F1
S315080042D01E93C023DB051F9312A8FEF707FB0028D1
S315080042E000D0FEE707230E93053B0F930023109398
S315080042F0119302210EA8FEF7BBFD002800D0FEE7A9
S31508004300022301930023039301A8FEF791FE0028D8
S3150800431000D0FEE721B000BD10B5FFF7A9FFFEF7F4
S315080043206FF9FFF7ADFF00F086F8FEF70FF910BD3D
S3150800433010B5FFF7F1FFFEF7A7F8FEF70FF9FEF73E
S3150800434001F9FAE7F0B58BB0254B1A6C0124224324
S315080043501A641A6C22400192019A5A6B22435A63D4
S315080043605A6B22400292029A5A6B022632435A63C9
S315080043705A6B32400392039ADA6B802189020A4308
S31508004380DA63DB6B0B400493049B002200210520B3
S315080043904042FEF75BF90022002102204042FEF768
S315080043A055F90022002101204042FEF74FF920234B
S315080043B005930694002507950895A027FF0505A9E6
S315080043C03800FEF7A7F90C23059306960795089576
S315080043D0099405A93800FEF79DF90BB0F0BDC04653
S315080043E0001002400D488546002103E00C4B5B583F
S315080043F0435004310B480C4B42189A42F6D30B4AE9
S3150800440002E0002313600432094B9A42F9D3FFF7FE
S3150800441027FF00F02DF8FFF78BFFFEE7009000203E
S3150800442050450008000000200C0000200C00002069
S3150800443008010020FEE710B5FEF7E0FDFA21890025
S31508004440FDF762FEFEF734F90420FEF74DF9002267
S31508004450002101204042FEF7F9F810BD10B5FEF71D
S31508004460EFF810BD10B5FEF7DFF8FEF74EF910BDF0
S3150800447070B500260C4D0D4C641BA410A64209D13C
S31508004480002600F021F80A4D0A4C641BA410A64227
S3150800449005D170BDB300EB5898470136EEE7B30077
S315080044A0EB5898470136F2E74845000848450008A2
S315080044B0484500084C45000803008218934200D17D
S315080044C0704719700133F9E7F8B5C046F8BC08BC5F
S315080044D09E467047F8B5C046F8BC08BC9E4670476D
S315080044E000000000000000000000000000000000BE
S315080044F000000000000000000000000000000000AE
S315080045000100000002000000030000000400000093
S31508004510060000000700000008000000090000006F
S31508004520000000000000000000000000000000007D
S315080045300100000002000000030000000400000063
S30D0800454020DDFF7F01000000E9
S30908004548E920000850
S3090800454CC120000874
S3110800455001000000040000000024F40034
S705080043E5CA
